:1000000042C036C665C064C063C062C061C060C023
:100010005FC05EC05DC05CC05BC05AC059C0090211
:1000200012000101008064090400000000000000CB
:1000300012011001FF000008C016DC0500010102DA
:1000400003011003420065007400610031002E00BE
:1000500031001603440047003800530041005100AE
:100060002D004900320043001A0377007700770023
:100070002E006F0062006400650076002E006100B3
:1000800074000403090411241FBECFE5D1E0DEBFD4
:10009000CDBF84B78093B40014BE88E10FB6F89446
:1000A00081BD11BC0FBE10E0A0E6B0E0E8EEFFE0BD
:1000B00003C0C89531960D92A636B107D1F710E06E
:1000C000A6E6B0E001C01D92A43BB107E1F738C439
:1000D00097CF01972FEF8F3F9207D9F70895B39BE2
:1000E000FECF08951092780087B3857F87BB8091FB
:1000F000610090916200EDDFF2DF87B38260877F5D
:1001000087BB8091610090916200E3DF87B38A60D2
:1001100087BB089587B38A6087BB80916100909107
:100120006200D7DF87B38260877F87BB80916100E1
:1001300090916200CEDFD3DF87B3857F87BB0895C0
:1001400087B38A6087BB8091610090916200C1DFB4
:1001500087B38260877F87BB809161009091620046
:10016000B8DFBDDF87B38A6087BB089587B3886037
:100170008D7F87BB8091610090916200AADF87B379
:10018000857F87BB8091610090916200A2DFA7DF2D
:1001900087B388608D7F87BB089587B388608D7F24
:1001A00087BB809161009091620093DF87B3857F68
:1001B00087BB80916100909162008BDF90DF86B3F6
:1001C00099278270907095958795982F87B388604E
:1001D0008D7F87BB892F992708950F931F93CF9306
:1001E000082F10E8C7E0812F802311F4A9DF01C098
:1001F000BDDF1695C150C7FFF6CFCFDF90917800D5
:10020000980F90937800CF911F910F9108951F93AD
:10021000CF9310E0C7E0110FC0DF182BC150C7FF0C
:10022000FACF8EDF812F9927CF911F9108951F93C9
:10023000CF9310E0C7E0110FB0DF182BC150C7FFFC
:10024000FACF94DF812F9927CF911F9108953F9284
:100250004F925F926F927F928F929F92AF92BF92D6
:10026000CF92DF92EF92FF920F931F93CF93DF9382
:10027000CDB7DEB728970FB6F894DEBF0FBECDBF5F
:100280004424A12CB12C10E3C12E11EBD12E60908F
:100290007000709071008090720090907300592DE2
:1002A000482D372D262DB3E0569547953795279540
:1002B000BA95D1F760E070E080E694EA5AD62983D7
:1002C0003A834B835C83ABE0FA2EE0906E00509053
:1002D0007E002F2D332789819A81732F622F33D689
:1002E000062F172F0F5F1F4F169507950330110527
:1002F00010F00E7F10700138110510F000E810E0CA
:100300002F2D33274427552701301105E1F0992D72
:10031000882D772D662D9695879577956795F8D5D5
:100320006D837E838F839887912F802F96958795F5
:10033000AA27BB27282F392F4A2F5B2F6D817E815B
:100340008F8198850FC0B92DA82D972D862D62E03D
:10035000B695A795979587956A95D1F7682F792FC8
:100360008A2F9B2FD5D56D837E838F83988780E0DE
:1003700090E02D813E814F8158852050304040498A
:10038000574910F081E090E020E030E04D815E813F
:100390006F817885A416B506C606D70610F021E051
:1003A00030E082239323892B41F081E0482EAD80F9
:1003B000BE80CF80D884E02E5F2CFA9480E090E05D
:1003C0005AE0F51611F481E090E020E030E068E0BA
:1003D000F61611F421E030E0822B932B892B09F0E3
:1003E000FA9473E07F1508F474CF50927E00E09287
:1003F0006E00442009F49BC0BD2DAC2D9B2D8A2D91
:1004000013E1B695A795979587951A95D1F780939F
:100410007A0090937B00A0937C00B0937D00EA94D7
:10042000E0926E008CEF580E50927E001092860083
:100430001092870010928800109289001092850017
:10044000F1E03F2E6090740070907500809076000F
:1004500090907700EE24FF240027112755249D2D2E
:100460008C2D7B2D6A2D592D482D372D262D81D58C
:10047000B52FA42F932F822F9AE1931548F0EE0CFD
:10048000FF1C001F111FE80EF11C011D111D02C0F1
:10049000550C580E9927AA27BB27592D482D372DC3
:1004A000262D682F792F8A2F9B2F32D5B92FA82F71
:1004B000972F862FA81AB90ACA0ADB0AAA0CBB1CF6
:1004C000CC1CDD1C3394A2E2A31548F650928500A3
:1004D000E0928600F09287000093880010938900D4
:1004E00065E0362EE4E8F0E0A5E8B0E08D91808389
:1004F00031973A94D9F7209180002F7330916E0094
:10050000832F992756E0880F991F5A95E1F7282BDA
:10051000209380003695369580917E00992745E09E
:10052000880F991F4A95E1F7382B30937F00842D6F
:10053000992728960FB6F894DEBF0FBECDBFDF9186
:10054000CF911F910F91FF90EF90DF90CF90BF90D0
:10055000AF909F908F907F906F905F904F903F9063
:100560000895C0DD80916F00880F37DE89E835DEA1
:1005700080E133DECFDD0895B5DD80916F00880F17
:100580002CDE89E82ADE80E028DEC4DD08950F93A2
:100590001F93CF93E6DFA6DD80916F00880F1DDEED
:1005A000809160001ADE0FE710E0C5E0F12FE02F28
:1005B00081910E2F1F2F11DEC150C7FFF7CFAADD8B
:1005C000DBDF90DD80916F00880F07DE87E805DEB6
:1005D00080E403DE9FDDCF911F910F910895A6E087
:1005E000B0E0EED4802D8F3F81F0EFE7F0E020E027
:1005F00030E095E0B32FA22F17968191082EE8D412
:1006000091502F5F3F4F97FFF5CF0895CF93DF9322
:10061000F92FE82F80917900803359F46630D0F1BA
:10062000AFE7B0E025E081918D93215027FFFBCF0C
:100630000FC0643078F1823371F4A0E7B0E023E0BA
:1006400081918D93215027FFFBCF01DE882311F18B
:10065000C6DF9DDF1FC08333E9F4CE2FDF2F40E0DC
:1006600050E023E0B52FA42F12968991082EB0D424
:1006700021504F5F5F4F27FFF5CFA1E0B0E080E052
:10068000082EA6D4A4E7B0E023E081918D932150F9
:1006900027FFFBCF81E090E0DF91CF9108950F938A
:1006A0001F93CF93DF93D92FC82F86E690E09093C6
:1006B0009900809398009981992339F48A818093D5
:1006C00066008B81809367008FC0913021F48A810E
:1006D0008A7F87BBD6C0923011F486B3E4C09330D2
:1006E00011F488B3E0C0943021F48A818A7F88BBFA
:1006F000C8C0953011F4F6DCC4C0963011F40ADDA0
:10070000C0C0973021F4109278008A8107C09830D9
:1007100049F4109278008A8160DD8B815EDD8091E2
:100720007800C1C0993051F4109278008A8155DD6B
:100730008B8153DD8C8151DD8D81F0CF9A3021F496
:10074000D1DC8A818E7F34C09B3019F4CBDC8A8166
:1007500041C09C3061F42A818B819927982F88278A
:10076000820F911D90936200809361008AC09F3038
:1007700009F4FFCF903149F42A818B819927B82F52
:10078000AA27A20FB11D8C817AC0913151F42A8120
:100790008B819927B82FAA27A20FB11D11D4802DC4
:1007A00082C0903251F49EDC8A81880F16DD8B81E5
:1007B00014DD8C8112DDAEDCB2CF9132C1F492DC5B
:1007C0008A81880F0ADD8B8108DD8CDC8A8199277C
:1007D000880F991F816001DD2ADD809367009ADC14
:1007E000809178008093660082E090E060C0923251
:1007F00029F48A8180936F00B4DE91CF933229F47B
:100800008A8180936F00B8DE8ACF892F805387302A
:1008100060F48A8180936F008B818093600089816E
:10082000809379008FEF90E042C09F3301F55ADC4E
:100830008A81880FD2DC87E0D0DC54DC8A8199275A
:10084000880F991F8160C9DC06E610E0C4E0DFDC98
:10085000F12FE02F81930E2F1F2FC150C7FFF7CF2D
:10086000E6DC80936B0056DC86E090E020C090349C
:1008700009F455CF913441F4A6E0B0E08A81082E06
:10088000A7D380E090E013C0903539F48A818823A3
:1008900011F4C49804C0C49A02C0913519F486B307
:1008A000827201C08FEF8093660081E090E0DF915B
:1008B000CF911F910F910895EF92FF920F931F9385
:1008C000CF9310E800E0C02FC10FC1BFBED129E017
:1008D000843392070CF40C2F1695A9F7C02FE82E3D
:1008E000F92EC150C1BFCF5F81B7282F33270C2FFE
:1008F0001127912F802F019682179307ACF0A5D175
:100900008453994097FF03C0909581959F4F8E1512
:100910009F051CF4E82EF92EC1B781B78F5F81BF08
:1009200081B7282F3327E5CFC1BFA0E0B0E081B762
:10093000082E4ED3CF911F910F91FF90EF90089505
:10094000CFE5D1E0DEBFCDBF80E096EFA8E4B2E70F
:100950008093740090937500A0937600B093770015
:10096000A1E0B0E02DD3802D8F3F81F0E4E7F0E0EF
:1009700020E030E043E0B32FA22F129621D3802D48
:10098000819341502F5F3F4F47FFF5CFA6E0B0E086
:1009900017D3802D992780936F008F3F89F0EFE761
:1009A000F0E020E030E045E0B32FA22F179608D307
:1009B000802D819341502F5F3F4F47FFF5CFE7DDFB
:1009C000A0E0B0E0FDD2802D282F33272F3F09F083
:1009D00021BFBA9AE3EBF1EF4BE38E2F9F2F0197E4
:1009E000F1F7415047FFF9CFBA9880E187BB18BAB9
:1009F00088E190E02BE00FB6F894A89581BD0FBE7A
:100A000021BD03D17894A89501D0FDCF1F93CF933A
:100A1000DF9360919A0016160CF092C080919700B7
:100A2000CAEAD0E0C81BD109635030E010E88091D9
:100A300096008D3209F06BC08AE5809363006830C0
:100A400009F078C08881807609F04EC083E990E093
:100A5000309393002981222321F43093940032E0D3
:100A60000FC0253021F48A8180939B0048C0263036
:100A700061F510EC8B81813041F480E390E032E14C
:100A800090939900809398003AC0823019F48EE1D7
:100A900090E0F5CF833099F58A81882321F482E8AC
:100AA00090E034E0EDCF813021F488E690E03AE147
:100AB000E7CF823021F482E590E036E1E1CF833068
:100AC000F1F482E490E030E1DBCF283019F48DE9D5
:100AD00090E008C0293021F48A8180939D000FC0E6
:100AE0002A3069F431E0CCCF8C2F9D2FD8DD382F00
:100AF0008F3F29F4888187FF1CC03E811AC08F81F7
:100B00008823C1F48E818317A8F4382F13C08091F5
:100B10006D0087FD0FC08C2F9D2F78DD3FEF831771
:100B200031F4309364008EE18093630002C0811140
:100B300030E010E010936D003093640010929A0042
:100B40008091630084FF44C0809164008F3F09F46A
:100B50003FC0682F893008F068E0861B80936400EE
:100B60001BE480916D0080FD13EC8F5F80936D001E
:100B7000ABE8B0E0E0919800F0919900962F915089
:100B800086FF08C09F3F61F0C895802D8D933196F8
:100B90009150F8CF9F3F21F081918D939150FACFE2
:100BA000F0939900E09398007727C62F693040F4BE
:100BB0008BE890E046D09C2F9C5FC83028F401C0A1
:100BC0009EE18FEF8093640010938A0090936300FE
:100BD0009AE086B3857011F49150D9F7992321F4E6
:100BE00090939B0090939500C0E0992309F4C1E095
:100BF00080916C008C1729F0CC2309F45DDEC09342
:100C00006C00DF91CF911F91089585B7836085BFF8
:100C10008BB780648BBF0895A82FB92F80E090E038
:100C200041E050EA60956F5F58F42D9138EF8227CC
:100C30009795879510F0842795273F5FC8F3F3CFEA
:100C40000895EADF8D939D930895A6E0882799275C
:100C5000AA9569F00197E1F3B299FCCFB29BFECF60
:100C600081E09927A6B3019611F0A570D9F70895F0
:100C7000CF93CFB7CF93B29BFECFB29B0BC0B29BAB
:100C800009C0B29B07C0B29B05C0B29B03C0B29B18
:100C900001C0D3C00F92DF93C0919700DD27C256E9
:100CA000DF4F012EB29B03C0DF910F90E6CF2F9351
:100CB0000F931F934F932FEF4F6F06B302FB20F953
:100CC0005F933F9350E03BE065C016B30126502987
:100CD00052FDC89556B3012702FB25F92F7306B3C1
:100CE000B1F05027102712FB26F906B22230F0F09F
:100CF00000C016B3012702FB27F90126502906B2CE
:100D00002430E8F54F77206816B30000F6CF50275F
:100D10004F7D206206B2102F000000C006B30026EF
:100D20005029102712FB26F906B2E2CF4F7B06B3FB
:100D3000206400C0DACF01265029157006B269F18F
:100D40004E7F2160012F16B328C0002650294D7F09
:100D500006B22260102F29C0012650294B7F06B20F
:100D60002460012F2DC016B301265029477F28602B
:100D7000000006B22EC04F7E06B3206130C042276D
:100D800006B3499300265029102706B24FEF12FBF5
:100D900020F9297F16B379F2157059F101265029EF
:100DA00006B2012702FB21F9237F06B371F2002668
:100DB00050293150D0F006B2102712FB22F9277EBD
:100DC00016B351F201265029012702FB06B223F97E
:100DD0002F7C49F2000006B3102712FB24F90026ED
:100DE000502906B22F7939F270CF10E41ABF0027CC
:100DF00017C03B503195C31BD04010E41ABF088187
:100E0000033CF9F00B34E9F0209195001981110FA2
:100E10001213EDCF093651F10D3211F0013E39F7C1
:100E200000939C003F915F914F911F910F912F91E3
:100E3000DF910F90CAB7C6FD1ECFCF91CFBFCF9124
:100E4000189500919C00002369F310919A001123DA
:100E500021F5343022F130939A00009396001091DE
:100E600097003BE0311B3093970019C000919A0026
:100E700001309CF40AE53091630034FD11C0009309
:100E80006300CAE8D0E010C0052710E000C021C010
:100E9000052710E0C89508BB14C03AE501C032ED43
:100EA000032EC0E0D0E032E017B31560C29A08B359
:100EB00017BB55E020E84FEF20FF052708BB27951B
:100EC00017951C3F28F700004552B0F720FF052773
:100ED000279508BB17951C3FB8F629913A9561F7FD
:100EE0000A7F10919B00110F08BBC250D04011F037
:100EF0001093950010E41ABF046017B31A7F402FB7
:100F00004A7F54E05A95F1F708BB17BB48BB8ACF1C
:100F1000FF27EE27BB27AA2760FF04C0A20FB31F3D
:100F2000E41FF51F220F331F441F551F9695879509
:100F30007795679589F70097760771F79F2F8E2F22
:100F40007B2F6A2F0895AA1BBB1B51E107C0AA1F64
:100F5000BB1FA617B70710F0A61BB70B881F991F5A
:100F60005A95A9F780959095682F792F8A2F9B2FF6
:100F70000895A1E21A2EAA1BBB1BEA2FFB2F0DC05E
:100F8000AA1FBB1FEE1FFF1FA217B307E407F50739
:100F900020F0A21BB30BE40BF50B661F771F881F15
:100FA000991F1A9469F76095709580959095262FF2
:100FB000372F482F592F6A2F7B2F8E2F9F2F089561
:100FC000E199FECFBFBBAEBBE09A11960DB208957A
:100FD000E199FECFBFBBAEBB0DBA11960FB6F89428
:080FE000E29AE19A0FBE0895A8
:060FE8000728005AFF007B
:00000001FF
